:100000000C948A010C943B290C943B290C943B29B9
:100010000C943B290C943B290C9452230C94782388
:100020000C943B290C943B290C943B290C943B29C0
:100030000C943B290C943B290C9428270C943B29C5
:100040000C943B290C943B290C943B290C943B29A0
:100050000C943B290C943B290C943B290C943B2990
:100060000C943B290C943B290C943B290C943B2980
:100070000C943B290C943B290C943B290C943B2970
:100080000C943B290C943B290C94101F0C943B2995
:100090000C943B290C943B290C943B290C943B2950
:1000A0000C943B290C943B290C943B290C943B2940
:1000B0000C943B290C943B290C943B290C943B2930
:1000C0000C943B290C943B290C943B290C943B2920
:1000D0000C943B290C943B290C943B290C943B2910
:1000E0000C943B290C943B290C941E210C94532115
:1000F0000C943B290C943B290C943B290C943B29F0
:100100000C943B290C943B290C943B290C94CD1F57
:100110000C943B290C943B290C943B290C943B29CF
:100120000C943B290C943B290C943B290C943B29BF
:100130000C943B290C943B290C943B290C943B29AF
:100140000C943B290C943B290C943B290C943B299F
:100150000C943B290C943B290C943B290C943B298F
:100160000C943B290C943B290C943B290C943B297F
:100170000C943B290C943B290C943B290C943B296F
:100180000C943B290C943B290C943B290C943B295F
:100190000C943B290C943B290C943B290C943B294F
:1001A0000C943B290C943B290C943B290C943B293F
:1001B0000C943B290C943B290C943B290C943B292F
:1001C0000C943B290C943B290C943B290C943B291F
:1001D0000C943B290C943B290C943B290C943B290F
:1001E0000C943B290C943B290C943B290C943B29FF
:1001F0000C943B290C943B290C943B2983108E10C2
:100200009410A410AD106111B61061116111DD10D0
:10021000611161116111F3106111611161116111BD
:10022000FE106111611138116111611161116111CB
:10023000611161116111C5106111611161115611D6
:10024000611161116111611161116111611161111E
:100250006111EA102F1161116111611161116111B8
:1002600061116111611161116111611161116111FE
:10027000611161116111BF1020002214802214232A
:10028000A300528423A32C59802C592C63005413AF
:100290002C632C6C802C6C2C7400541D2C742C98AA
:1002A000802C982C9900054D2C992C9A0054252CC3
:1002B0009A2CA5802CA52CA60054262CA62CAC800C
:1002C0000C94FE100C9494100C9438110C94DD10C6
:1002D0000C9461110C9424280C94B6100C94EE200C
:1002E0000C94EA100C94DF0C0C94FA210C942F114E
:1002F0000C9456110C94C5100C94AD020C94AD10D6
:100300000C94BF100C94F3100C94A4100C94831054
:100310000C948E1011241FBECFEFCDBFDFE3DEBFE4
:1003200000E00CBF18BE19BE1ABE1BBEE8E7F2E023
:1003300042E019C0B791A79137912791079107FD26
:100340000EC097918791EF01F92FE82F0BBF07900F
:100350000D92A217B307D9F7FE011BBE04C01D9270
:10036000A217B307E1F7E03CF40721F71BBE0E9498
:0A03700007200C94D627F894FFCF65
:10037A0083F9A200444E6E00FC291500D1572700CC
:10038A00DD34F50062DBC0003C99950041904300E2
:10039A006351FE00BBDEAB00B761C5003A6E2400B4
:1003AA00D24D42004906E00009EA2E001C92D10013
:1003BA00EB1DFE0029B11C00E83EA700F5358200BE
:1003CA0044BB2E009CE98400B4267000417E5F0085
:1003DA00D6913900538339009CF439008B5F84002D
:1003EA0028F9BD00F81F3B00DEFF97000F980500B3
:1003FA00112FEF000A5A8B006D1F6D00CF7E360059
:10040A0009CB2700464FB7009E663F002DEA5F00E2
:10041A00BA277500E5EBC7003D7BF100F739070005
:10042A0092528A00FB6BEA001FB15F00085D8D00E3
:10043A00300356007BFC4600F0AB6B0020BCCF00BB
:10044A0036F49A00E3A91D005E619100081BE600DC
:10045A0085996500A0145F008D40680080D8FF0070
:10046A0027734D0006063100CA561500C9A8730045
:08047A007BE260006B8CC00006
:100482000200530300000700000F000010000F11CC
:10049200008C12000F13008C14008C15008C1600B7
:1004A2008C17008C1A00001B00011C00001D00109C
:1004B2001E00001F00002000002100002A00002B67
:1004C20000012C00002D00102E00002F0000300033
:1004D200003100003A00003B00853C00003D001A5C
:1004E2003E00323F00004000004100065A00005B1F
:1004F2000000950000960000970000980000990007
:10050200009A00009B0000A20000A30000A40000CB
:03051200B700929D
:10051500DA0FC93F6821A233C434C2278B62C61BD8
:100525001CDC800F0229D10314000000000000002C
:0C0535001F1E1F1E1F1F1E1F1E1F1F1D4C
:080541000300040004000600A1
:04054900474D5400C6
:01054D0001AC
:10054E00A2E7B1E0EDEAF2E00C945225C959DE4F74
:10055E008883C756D140C859DE4F9883C856D140BC
:10056E00C35ADE4F68837983CD55D1407A01C75B7C
:10057E00DE4F28833983C954D140CD59DE4F0883CD
:10058E001983C356D140C801880F991F092E000C3C
:10059E00AA0B8F5B9A4FAF4FFC015A2F0E94FF2779
:1005AE004B01770FAA08BB08CB5ADE4F888299827F
:1005BE00AA82BB82C555D140C90101975C01990F32
:1005CE00CC08DD08CF5ADE4FA882B982CA82DB8200
:1005DE00C155D140C701039768E170E00E943326F0
:1005EE0077FD0DC04B01770FAA08BB08C75ADE4F27
:1005FE0088829982AA82BB82C955D14008C0C75A47
:10060E00DE4F188219821A821B82C955D140A8EE7C
:10061E00BFEFC75ADE4F288139814A815B81C955A8
:10062E00D1402F5F3F4F4F4F5F4F0E946C28870185
:10063E00FF0C220B330B5B016C01A00EB11EC21E10
:10064E00D31ECF5BDE4FA882B982CA82DB82C15431
:10065E00D140C75ADE4F488059806A807B80C95589
:10066E00D140CF5ADE4FC880D980EA80FB80C15579
:10067E00D1404C185D086E087F08CB5ADE4F88803B
:10068E009980AA80BB80C555D1408C0C9D1CAE1C98
:10069E00BF1CCB5BDE4F88829982AA82BB82C55477
:1006AE00D1408E010F551F4F6201CC0CDD1CCC0CBE
:1006BE00DD1CC601DD0CAA0B9C014A2F26583C4FAF
:1006CE004F4F6901E42E812C912C5401CB5BDE4FF0
:1006DE00288139814A815B81C554D140281539055D
:1006EE004A055B0514F1D501C401840D951DA61DA7
:1006FE00B71DB7FD07C0F6015E2D0E9472270E943E
:10070E00921F03C060E070E0CB01D8016D937D9322
:10071E008D939D938D01BFEF8B1A9B0AAB0ABB0A7B
:10072E00E4E0CE0ED11CE11CD1CF8E010F5F1F4F26
:10073E00C35BDE4F08831983CD54D140C75BDE4FB8
:10074E0088809980C954D140C401990CAA0BBB0B67
:10075E000197A109B1095C01AA0CBB1CAA0CBB1C18
:10076E00C15ADE4FA882B982CF55D140212C312CEF
:10077E00412C512C3201CB5ADE4F88809980AA80B1
:10078E00BB80C555D14084149504A604B7040CF45F
:10079E0084C0C959DE4F9880C756D140CB5BDE4F1F
:1007AE009882C554D140C859DE4FA880C856D14052
:1007BE00CA5BDE4FA882C654D140C15ADE4FC880F4
:1007CE00D980CF55D140C20CD31CCB59DE4FC88235
:1007DE00D982C556D14000E010E0812C912C5401F5
:1007EE00C12CD12C7601CF5ADE4F288139814A8116
:1007FE005B81C155D1402C153D054E055F05A4F119
:10080E00CB59DE4FE881F981C556D140E00FF11F7B
:10081E0021EA30E02C0F3D1FE20FF31FCB5BDE4FC2
:10082E00A881B981C554D1402D913D914D915D91D5
:10083E00CB5BDE4FA883B983C554D14060817181F3
:10084E00828193810E941B299B01AC01C501B401D9
:10085E000E9497284B015C01BFEFCB1ADB0AEB0A13
:10086E00FB0A04501109BFCFC35BDE4FA881B981CB
:10087E00CD54D1408D929D92AD92BD92C35BDE4F11
:10088E00A883B983CD54D140BFEF4B1A5B0A6B0AD4
:10089E007B0AE4E02E0E311C6ECFCB5ADE4F8881E0
:1008AE009981AA81BB81C555D1400197A109B10992
:1008BE007C01EE0CFF1CEE0CFF1CC359DE4FE882D0
:1008CE00F982CD56D140CB5ADE4F488059806A808E
:1008DE007B80C555D14088E190E08C01CF5BDE4F27
:1008EE0028813981C154D140021B130BCB59DE4FE5
:1008FE0008831983C556D140C75BDE4F8881998125
:10090E00C954D14001974C01990FAA08BB08C1598F
:10091E00DE4F88829982AA82BB82CF56D140520185
:10092E00AA0CBB1CAA0CBB1CC35BDE4FA882B982EF
:10093E00CD54D140E1E0F0E0EC0FFD1FEA0DFB1DC0
:10094E00C080D180E280F3801E0101EF200E311CA9
:10095E00D301C2010197A109B1094C01880C991C60
:10096E00880C991CC15ADE4F88829982CF55D1408E
:10097E00CB5BDE4F28823982C554D14053014201F0
:10098E0000E010E0181419041A041B040CF059C0EE
:10099E0020E030E040E853E3C701B6010E941B2976
:1009AE000E94B2280E94921FC75BDE4F6883798334
:1009BE008A839B83C954D14020E030E040E85BE459
:1009CE000E941B299B01AC01C701B6010E9496280B
:1009DE000E94B228CB5BDE4FA881B981C554D140AD
:1009EE006D937D938D939D93CB5BDE4FA883B983DF
:1009FE00C554D140B1E08B1A9108A108B108C15A73
:100A0E00DE4FE881F981CF55D140E00FF11FCC24A4
:100A1E00C394D12CCC0EDD1EEC0DFD1D2081318139
:100A2E0042815381C75BDE4F688179818A819B81C8
:100A3E00C954D1400E9497286B017C0104501109C2
:100A4E00A1CFCF5BDE4F08811981C154D140A801DF
:100A5E00C701B6010E94E61C6B017C0120E030E06C
:100A6E0040E05EE30E941B290E94FA1520E030E070
:100A7E0040E051E40E941B299B01AC01C701B60165
:100A8E000E9496286B017C010E94B228C75BDE4F44
:100A9E00688379838A839B83C954D1400E94921FB5
:100AAE009B01AC01C701B6010E9496286B017C0127
:100ABE00CF5BDE4F88809980AA80BB80C154D14025
:100ACE00181419041A041B040CF05DC0D301C201E2
:100ADE000197A109B109880F991F880F991FE1EF9E
:100AEE00F0E0EC0FFD1FE80FF91F4081518162818C
:100AFE0073814A015B01CB59DE4F0880C556D14048
:100B0E0004C0B594A794979487940A94D2F7C75BC0
:100B1E00DE4F88819981AA81BB81C954D140880D4D
:100B2E00991DAA1DBB1DC75BDE4F88839983AA83BF
:100B3E00BB83C954D140CB59DE4F0880C556D14036
:100B4E0004C0880C991CAA1CBB1C0A94D2F7481925
:100B5E0059096A097B09408351836283738387E154
:100B6E0090E0CF5BDE4FA881B981C154D1408A1B82
:100B7E009B0B4A015B0104C0B594A794979487948C
:100B8E008A95D2F728C0CF5BDE4F88809980AA80E5
:100B9E00BB80C154D14089288A288B2891F5D30176
:100BAE00C2010197A109B109880F991F880F991FDA
:100BBE00E1EFF0E0EC0FFD1FE80FF91F808191814E
:100BCE00A281B3814C015D0157E1B594A79497942E
:100BDE0087945A95D1F7CB5BDE4F88829982AA8291
:100BEE00BB82C554D140CB5BDE4F88809980AA80F2
:100BFE00BB80C554D140181419041A041B04FCF010
:100C0E00E2C020E030E040E05FE30E94F02887FF82
:100C1E0009C0CB5BDE4F188219821A821B82C55423
:100C2E00D140D1C032E0832E912CA12CB12CCB5BC4
:100C3E00DE4F88829982AA82BB82C554D140C75B9F
:100C4E00DE4F288139814A815B81C954D1402F5FA3
:100C5E003F4F4F4F5F4FC75BDE4F288339834A8329
:100C6E005B83C954D14080E090E0DC01812C912C53
:100C7E00540184159505A605B705ACF5F101408123
:100C8E0051816281738181149104A104B10481F4B4
:100C9E004115510561057105F9F0812C912C540116
:100CAE00B394841A950AA60AB70AB501A4010CC01A
:100CBE0088248A94982CA82CB12C841A950AA60AFA
:100CCE00B70AB501A401F101408351836283738396
:100CDE00812C912C540183940196A11DB11DF4E039
:100CEE002F0E311CC6CFCF5BDE4F288139814A8152
:100CFE005B81C154D1401216130614061506CCF5AD
:100D0E002130310541055105D9F02230310541051B
:100D1E00510579F5D301C2010197A109B109880FD7
:100D2E00991F880F991FE1EFF0E0EC0FFD1FE80F00
:100D3E00F91F40815181628173816F73772715C0CE
:100D4E00D301C2010197A109B109880F991F880F1C
:100D5E00991FE1EFF0E0EC0FFD1FE80FF91F408146
:100D6E005181628173816F777727408351836283CC
:100D7E007383CB5BDE4F488159816A817B81C55479
:100D8E00D1404230510561057105E9F4A701960184
:100D9E0060E070E080E89FE30E9496286B017C0182
:100DAE0089288A288B2879F0A80160E070E080E815
:100DBE009FE30E94E61C9B01AC01C701B6010E9495
:100DCE0096286B017C0120E030E0A901C701B60135
:100DDE000E94EB288111CFC17301620151E0C51A47
:100DEE00D108E108F108B301A20120E030E080E073
:100DFE0090E0DC014150510961097109CB5ADE4F77
:100E0E0088809980AA80BB80C555D1404815590568
:100E1E006A057B05D4F0C15ADE4FE881F981CF55C2
:100E2E00D140E20FF31F11EF812E912C8C0E9D1EDF
:100E3E00E80DF91D80809180A280B38088299929C0
:100E4E00AA29BB2924503109D5CF892B8A2B8B2B6C
:100E5E0009F046C180E090E041E050E060E070E0D3
:100E6E000497C359DE4FE881F981CD56D140E80F82
:100E7E00F91F21EFA22EB12CAC0EBD1EEA0DFB1DEB
:100E8E000481158126813781012B022B032B29F436
:100E9E004F5F5F4F6F4F7F4FE3CF530142010FEF15
:100EAE00801A900AA00AB00AC75ADE4FC880D980AD
:100EBE00EA80FB80C955D140C80CD91CEA1CFB1C2A
:100ECE00CC0CDD1CCC0CDD1CC601DD0CAA0B8C0180
:100EDE002A2F06581C4F2F4F6801E22EC159DE4FA4
:100EEE0088819981AA81BB81CF56D140880D991DE9
:100EFE00AA1DBB1D8C01000F111F000F111FC5591C
:100F0E00DE4F08831983CB56D1408401000F111F89
:100F1E00000F111FC759DE4F08831983C956D140E0
:100F2E00212C312CD301C201840F951FA61FB71F90
:100F3E00C15ADE4F88839983AA83BB83CF55D14094
:100F4E00C15ADE4F088119812A813B81CF55D1408C
:100F5E00081519052A053B050CF4BFC0C559DE4F0F
:100F6E0008811981CB56D140020D131DC35BDE4F94
:100F7E0008831983CD54D14001EA10E00C0F1D1FD8
:100F8E00C35BDE4F28813981CD54D140020F131F30
:100F9E00F6015E2D0E9472270E94921FD8016D935A
:100FAE007D938D939C931397C959DE4FF880C75646
:100FBE00D140CB5BDE4FF882C554D140C859DE4FCD
:100FCE00F880C856D140CA5BDE4FF882C654D14075
:100FDE00C75BDE4F188219821A821B82C954D14018
:100FEE0000E010E0412C512C3201C75BDE4F4881EE
:100FFE0059816A817B81C954D140CF5ADE4F888195
:10100E009981AA81BB81C155D14084179507A60746
:10101E00B7070CF443C0C35BDE4FE881F981CD54B2
:10102E00D140E00FF11F21EA30E02C0F3D1FE20FFF
:10103E00F31FCB5BDE4FA881B981C554D1402D91F2
:10104E003D914D915D91CB5BDE4FA883B983C55425
:10105E00D14060817181828193810E941B299B0105
:10106E00AC01C301B2010E9497282B013C01C75B62
:10107E00DE4F288139814A815B81C954D1402F5F6F
:10108E003F4F4F4F5F4FC75BDE4F288339834A83F5
:10109E005B83C954D14004501109A7CFC759DE4F05
:1010AE00E881F981C956D140E20DF31DA1E0B0E00F
:1010BE00AC0FBD1FEA0FFB1F40825182628273820A
:1010CE00BFEF8B1A9B0AAB0ABB0AE4E02E0E311C53
:1010DE00F4E0CF0ED11CE11C33CF280139011FCC17
:1010EE00CF5BDE4F288139814A815B81C154D1406B
:1010FE002851310941095109CF5BDE4F28833983CD
:10110E004A835B83C154D140C601880F991F880F53
:10111E00991F2601370120E030E024503109F901F2
:10112E00E80FF91F61EF70E06C0F7D1FE60FF71FE0
:10113E004481558166817781452B462B472B09F0DB
:10114E009EC041E0441A510861087108CF5BDE4F22
:10115E00488159816A817B81C154D14048515109DE
:10116E0061097109CF5BDE4F488359836A837B83A4
:10117E00C154D140D2CFCF5BDE4F48815981C1548B
:10118E00D140519541955109C701B6010E94E61C07
:10119E006B017C0120E030E040E85BE40E94F02827
:1011AE0087FD57C020E030E040E853E3C701B601A9
:1011BE000E941B290E94B2280E94921F4B015C01C3
:1011CE0001EF10E00C0F1D1FC35BDE4F888199816C
:1011DE00CD54D140080F191F20E030E040E85BE409
:1011EE00C501B4010E941B299B01AC01C701B601C8
:1011FE000E9496280E94B228D8016D937D938D93FC
:10120E009C931397BFEF4B1A5B0A6B0A7B0ACF5B5B
:10121E00DE4F088119812A813B81C154D140085E7D
:10122E001F4F2F4F3F4FCF5BDE4F088319832A830B
:10123E003B83C154D1408201000F111F000F111FBB
:10124E0021EF30E02C0F3D1F020F131FC501B4011B
:10125E000EC001EF10E00C0F1D1FC35BDE4F888028
:10126E009980CD54D140080D191DC701B6010E94B9
:10127E00B228D8016D937D938D939C931397CF5B7A
:10128E00DE4F48815981C154D14060E070E080E862
:10129E009FE30E94E61C4B015C01C15ADE4F48825F
:1012AE005982CF55D1401201220C331C220C331C13
:1012BE007301620100E010E0F7FC3CC0C801820D32
:1012CE00931DE1E0F0E0EC0FFD1FE80FF91FCF5B7F
:1012DE00DE4FE883F983C154D140E1EFF0E0EC0F2B
:1012EE00FD1FE80FF91F60817181828193810E9439
:1012FE00921FA50194010E941B29CF5BDE4FA8818E
:10130E00B981C154D1406D937D938D939C93139766
:10131E0020E030E040E853E3C501B4010E941B29F0
:10132E004B015C01B1E0CB1AD108E108F108045081
:10133E001109C2CF8E010F5A1F4FC35BDE4F0883B8
:10134E001983CD54D140CF5BDE4F188219821A8299
:10135E001B82C154D140CF5ADE4F18821982C1551B
:10136E00D140D301C201CF5BDE4F88809980AA8025
:10137E00BB80C154D14088199909AA09BB09B7FD90
:10138E00B2C075E1872E75E0972E70E0A72E610131
:10139E00CF5ADE4FE880F980C155D140CE18DF0814
:1013AE00CB59DE4FC882D982C556D14000E010E03D
:1013BE00C75ADE4F188219821A821B82C955D14034
:1013CE00C12CD12C7601CB5ADE4F688179818A816E
:1013DE009B81C555D1406C157D058E059F050CF47E
:1013EE0047C0CF5BDE4F88819981AA81BB81C154F2
:1013FE00D1408C159D05AE05BF05D4F1CB59DE4FFE
:10140E00A881B981C556D140A00FB11F21E030E0AF
:10141E002C0F3D1FA20FB31FF4015A2D0E947227ED
:10142E009B01AC016D917D918D919C910E941B2928
:10143E009B01AC01C75ADE4F688179818A819B81FD
:10144E00C955D1400E949728C75ADE4F68837983C9
:10145E008A839B83C955D1403FEFC31AD30AE30A4F
:10146E00F30A44E0840E911CA11C0C5F1F4FABCFFE
:10147E00C35BDE4FA881B981CD54D140C75ADE4F30
:10148E0088809980AA80BB80C955D1408D929D924B
:10149E00AD92BD92C35BDE4FA883B983CD54D140CC
:1014AE00CF5ADE4F08811981C155D1400C5F1F4FB5
:1014BE00CF5ADE4F08831983C155D140CF5BDE4F23
:1014CE00288139814A815B81C154D1402F5F3F4FC2
:1014DE004F4F5F4FCF5BDE4F288339834A835B8349
:1014EE00C154D1403ECFCD59DE4F08811981C3562C
:1014FE00D1400330110574F4013011050CF048C0D1
:10150E000115110509F041C200E010E060E070E045
:10151E00CB0146C0CD59DE4F08811981C356D1404B
:10152E000330110509F031C251E5852E912C8C0E38
:10153E009D1E820C931CCF5BDE4F88829982C15414
:10154E00D14014012CEFC15ADE4F08811981CF55BD
:10155E00D14020034001219F900C1124CD59DE4F24
:10156E0088829982C356D140D301C2010197A10945
:10157E00B1095C01AA0CBB1CAA0CBB1CC75ADE4FDE
:10158E00A882B982C955D140810173016201B0C0F0
:10159E007301620100E010E060E070E0CB0135C045
:1015AE0077FC18C0F101E00FF11F41E5C42ED12CDC
:1015BE00CC0EDD1EEC0DFD1D20813181428153814B
:1015CE000E94972821E0421A5108610871080450C0
:1015DE001109E6CFCB5BDE4F88809980AA80BB8055
:1015EE00C554D140DC01CB0181149104A104B10496
:1015FE0009F0B058C35ADE4FE881F981CD55D1407C
:10160E0080839183A283B383C0C1F7FC18C0F1011C
:10161E00E00FF11F31E5832E912C8C0E9D1EE80DEF
:10162E00F91D20813181428153810E94972821E04A
:10163E00C21AD108E108F10804501109E6CFCB5BBC
:10164E00DE4F88809980AA80BB80C554D1408B0123
:10165E009C0189288A288B2809F03058C35ADE4FFE
:10166E00A881B981CD55D1400D931D932D933C93F7
:10167E0013979B01AC018E010F5A1F4FF801619118
:10168E007191819191918F010E949628C12CD12C3C
:10169E007601C3944C145D046E047F0474F0D8017B
:1016AE002D913D914D915D918D010E949728BFEF37
:1016BE00CB1ADB0AEB0AFB0AEDCFCB5BDE4F888041
:1016CE009980AA80BB80C554D140DC01CB01811426
:1016DE009104A104B10409F0B058C35ADE4FE88159
:1016EE00F981CD55D14084839583A683B7834DC1AF
:1016FE001C141D041E041F040CF06DC0F1E0CF1A63
:10170E00D108E108F108CD59DE4F88819981C35681
:10171E00D140800F911FC75ADE4F88809980C955DE
:10172E00D140880E991ECF5ADE4F88829982C155BC
:10173E00D140D4018D909D90AD90BC90CB5ADE4F90
:10174E0088829982AA82BB82C555D140F8018080D9
:10175E009180A280B380A5019401CB5ADE4F68819F
:10176E0079818A819B81C555D1400E949728C35BA0
:10177E00DE4F688379838A839B83CD54D1409B014E
:10178E00AC01CB5ADE4F688179818A819B81C55528
:10179E00D1400E949628A50194010E949728D80155
:1017AE006D937D938D939C931397C35BDE4F8880CF
:1017BE009980AA80BB80CD54D140CF5ADE4FA881EC
:1017CE00B981C155D1408D929D92AD92BC92139725
:1017DE00045011098DCF73016201E2E0CE16D104DF
:1017EE00E104F1040CF463C0B1E0CB1AD108E108B6
:1017FE00F108CD59DE4F08811981C356D140020D33
:10180E00131DC75ADE4F88809980C955D140080DE7
:10181E00191DD8018D909D90AD90BC90CB5ADE4F86
:10182E0088829982AA82BB82C555D140F1018080FF
:10183E009180A280B380A5019401CB5ADE4F6881BE
:10184E0079818A819B81C555D1400E949728CF5AB4
:10185E00DE4F688379838A839B83C155D1409B0178
:10186E00AC01CB5ADE4F688179818A819B81C55547
:10187E00D1400E949628A50194010E949728D1017B
:10188E006D937D938D939C931397CF5ADE4F8880E3
:10189E009980AA80BB80C155D140D8018D929D926E
:1018AE00AD92BC921397B4E02B1A310896CF00E09C
:1018BE0010E060E070E0CB0122E0421651046104BA
:1018CE007104B4F0CF5BDE4FE881F981C154D14091
:1018DE00E00FF11F20813181428153810E949728B0
:1018EE00F1E04F1A51086108710804501109E4CF54
:1018FE00CB5BDE4F88809980AA80BB80C554D140D7
:10190E0065960CAD1DAD2EAD3FAD6597811491045E
:10191E00A104B104E9F4C35ADE4FA881B981CD55B3
:10192E00D1400D931D932D933C93139769960CAD57
:10193E001DAD2EAD3FAD6997FD0104831583268342
:10194E00378318966D937D938D939C931B971DC033
:10195E003058C35ADE4FE881F981CD55D14000830E
:10196E0011832283338369960CAD1DAD2EAD3FAD31
:10197E00699730580483158326833783DC01CB01A6
:10198E00B05880879187A287B387C75BDE4F888167
:10199E009981C954D14087709927CE58DE4FE2E124
:0419AE000C949C25D4
:1019B200A6E1B0E0EFEDFCE00C9452257901D42EC3
:1019C200C52EB62FA72FF82FB92E40585D4B6E406B
:1019D2007F4F8F4F9F4F21153B474D415348624EDA
:1019E20071408105910511F008F008C20F87188B2C
:1019F2009B2D8F2F7A2F6B2F5C2D4D2D9701205809
:101A02003D454C4B584361097109810991091901FE
:101A12004D8359876D877983898B9A8BF0E8AF2E36
:101A2200A1E5BA2ECC24C394D12CE12CF12C00E0F8
:101A320010E00E94EE2129013A014B018E8B9B8B13
:101A420091014D8159856D85798189899A890E9493
:101A5200EC212D833E834F8358878D819E81AF81F8
:101A6200B885B7FF15C080589E4AAE4FBF4F8D83D1
:101A72009E83AF83B8879201A301B4018E899B89AB
:101A8200AFEF0E94BF2729013A014B018E8B9B8B3E
:101A92009201A301B4018E899B89A3E00E94BF2712
:101AA200E7E0AE2EB12CC12CD12CE12CF12C00E0C0
:101AB20010E00E94EC212D873E87AD85BE85B7FFE1
:101AC20003C01796AD87BE8751EBA52E6AE3B62EEB
:101AD20072E0C72ED12CE12CF12C00E010E0920133
:101AE200A301B4018E899B890E94EE2129873A873E
:101AF2004B875C879201A301B4018E899B890E9466
:101B0200EC21822E932EA42EB52EB7FE12C0B1EB7D
:101B12008B0EBAE39B1EB2E0AB1EB11C89859A857F
:101B2200AB85BC850197A109B10989879A87AB87E3
:101B3200BC87C501B4012CEA3EE840E050E00E94B7
:101B4200B42569017A01243031054105510529F492
:101B520043E0C42ED12CE12CF12CA4E5B1E7A7017E
:101B620096010E946C282B013C01480C591C6A1CEE
:101B72007B1CC301B20125EB35E040E050E00E943E
:101B8200B42549015A01293131054105510529F48C
:101B920038E1832E912CA12CB12CABE4BAEFA50134
:101BA20094010E946C28460E571E681E791EC301BE
:101BB200B2012DE631E040E050E00E94B4252983D5
:101BC2003A834B835C83243031054105510541F44E
:101BD20083E090E0A0E0B0E089839A83AB83BC838A
:101BE200A3E9BEEF29813A814B815C810E946C2876
:101BF200460E571E681E791E232B242B252B81F49B
:101C020081149104A104B10471F431E020E0C11403
:101C1200D104E104F10409F030E0832F922F05C0D2
:101C220080E090E002C081E090E01201ABE32A0E76
:101C3200311C280E391E9C0124593E4F22153305B2
:101C420024F483599E4F281A390A92E0880C991C71
:101C5200AA1CBB1C9A95D1F789819A81AB81BC8160
:101C6200880E991EAA1EBB1EA4E6B0E0A70196012B
:101C72000E94CB27860E971EA81EB91ED501C4014D
:101C8200BB0F880B982FDC0189839A83AB83BC83BB
:101C920069857A858B859C8520E931E040E050E0BA
:101CA2000E945527F22FE32F6A017B018C019401D8
:101CB200A5016981762F862F962FAF2EBE2E0E9408
:101CC2003F2849015A016B017C0125E335E040E0E0
:101CD20019821A82F901542F0E947128862F660FE9
:101CE200990BAA0BBB0B2F5F3F4F4F4F481659065C
:101CF2006A067B0654F0481A590A6A0A7B0AA981C5
:101D0200BA811196A983BA83E5CFE981FA81EA30D3
:101D1200F10574F03C97E983FA839401A501B601B9
:101D2200C701A1E00E94BF2749015A016B017C0152
:101D32009401A501B601C7012C593F474F4F5F4F90
:101D42006F4F7F4F8F4F9F4F2F3F3F4F41055105A1
:101D5200610571058105910511F008F04FC024E677
:101D6200820E911CAF85B8891A968D929C921B9710
:101D7200E981FA8132961896ED93FC931997FFEF59
:101D82004F1A5F0A16964D925C9217978D859E8523
:101D92001C968D939C931D971E962D923C921F9795
:101DA2006D817E818F81988520E13EE040E050E0A8
:101DB2000E94B425AF85B88914962D933C9315974C
:101DC2008CE3C82ED12CE12CF12C6D817E818F8188
:101DD2009885A70196010E94B4254B015C01CA01B6
:101DE200B901A70196010E94B425EF85F8896283A3
:101DF20073838082918280E090E002C08FEF9FEF38
:081E02006696E2E10C949C25B8
:101E0A004F925F926F927F928F929F92AF92BF9200
:101E1A00CF92DF92EF92FF92CF93DF9300D00F928F
:101E2A00CDB7DEB75C0169834A019C01ABEABAEA25
:101E3A000E94462796958795929582958F70892755
:101E4A009F708927BC0180E090E00E94901F9B014F
:101E5A00AC0166E57EE089EC90E40E9417292B012B
:101E6A003C01B50180E090E00E94901F9B01AC010B
:101E7A0066E57EE089EC90E40E9417296B017C01FB
:101E8A008981811120C0B40180E090E00E94901FF6
:101E9A004B015C019B01AC01C301B2010E941B29E9
:101EAA000E9482112B013C01A5019401C701B601D0
:101EBA000E941B290E9482119B01AC01C301B2013D
:101ECA000E941B29D0C08981813009F04AC0B4011F
:101EDA0080E090E00E94901F4B015C019B01AC01E5
:101EEA00C301B2010E941B290E94821169837A836D
:101EFA008B839C8320E030E040EC5FE3C701B601AE
:101F0A000E941B299B01AC01C501B4010E941B2937
:101F1A000E9482112DEC3CEC4CEC5EE30E941B29E2
:101F2A002B013C0120E030E040E05FE3C701B6014D
:101F3A000E941B299B01AC01C501B4010E941B2907
:101F4A000E9482119B01AC01C301B2010E94972831
:101F5A009B01AC0169817A818B819C810E941B293A
:101F6A0082C08981823009F051C0B40180E090E0DA
:101F7A000E94901F9B01AC01C301B2010E941B2960
:101F8A000E94821169837A838B839C83B501680DD1
:101F9A00791D80E090E00E94901F4B015C0120E0D7
:101FAA0030E040EC5FE3C701B6010E941B299B01A8
:101FBA00AC01C501B4010E941B290E9482112DECBB
:101FCA003CEC4CEC5EE30E941B292B013C0120E017
:101FDA0030E040E05FE3C701B6010E941B299B0184
:101FEA00AC01C501B4010E941B290E9482119B0108
:101FFA00AC01C301B2010E9497289B01AC0169811F
:10200A007A818B819C810E941B292DC08981833012
:10201A0039F5B40180E090E00E94901F9B01AC0169
:10202A00C301B2010E941B290E9482112B013C01AB
:10203A00B50176956795680D791D80E090E00E945C
:10204A00901F9B01AC01C701B6010E941B290E9487
:10205A0082119B01AC01C301B2010E941B2903C07A
:10206A0060E070E0CB012496CDBFDEBFDF91CF9157
:10207A00FF90EF90DF90CF90BF90AF909F908F909E
:0A208A007F906F905F904F900895D3
:10209400EF92FF920F931F93CF93DF93CDB7DEB7E9
:1020A400E497CDBFDEBFDC018C9190E0982F8827A8
:1020B40011962C911197822B23E43CE2F901808341
:1020C400918312968C911297828313969C91139705
:1020D4009383FD01E90FF11D8581F901828714962F
:1020E4004C911497448350E0FA013197EE33F10593
:1020F40008F0E5C08D018827E250FF4F8F4F0C9404
:102104002D28FD01878190E0982F88272085822B38
:102114000E94E12880E0EAC0CD0107960E94722463
:1021240080E0E4C0FD018781843008F0CAC081FBEF
:10213400112710F981700E94B327812F0E94292949
:1021440080E0D4C0FD018781833008F0BCC00E94C8
:102154002F2980E0CBC0FD018781833008F0B5C012
:102164000E942C2980E0C2C0FD018781803208F0E2
:10217400AEC00E94262980E0B9C0CD0107960E9416
:102184007C2280E0B3C0FD011581163008F0A1C0A7
:10219400111102C00E94DC28113011F40E94922413
:1021A400133011F40E948026153009F094C00E9467
:1021B400922680E09BC0892F90E005978234910598
:1021C4000CF08BC0CD0109960E943F1D80E08EC0AB
:1021D400FD018581843008F082C00E94E62880E0F9
:1021E40085C0FD01858190E0982F88272681822B68
:1021F4000E941B2880E07AC040911020413E08F4E0
:1022040070C0405E84E089834A8320E00FC0822F3F
:1022140090E0FC013B96E00FF11F3081E3E0F0E039
:10222400EC0FFD1FE80FF91F30832F5F241778F39D
:102234008DB79EB7C4978DBF9EBFADB7BEB711967D
:1022440084E3FE01319601900D928A95E1F70E9494
:102254005B26CDBFDEBF80E049C0FD0181858430AF
:1022640008F041C00E94E92480E040C0FD01838160
:102274009FEF980F9C3FC8F50F2EFDEFEF2EF02D2A
:10228400E80EF12C0AC0EF2DF0E03796E00FF11FB5
:1022940060818F2D0E94C528F394FE14A0F38E2D27
:1022A4000E94352980E022C0FD01858190E0982FAD
:1022B40088272681822B0E94592880E017C080E05D
:1022C40015C086E013C086E011C086E00FC086E02A
:1022D4000DC086E00BC080E009C087E007C086E03F
:1022E40005C086E003C086E001C086E0E496CDBF69
:1022F400DEBFDF91CF911F910F91FF90EF90089572
:10230400CF92DF92EF92FF92CF93DF9300D00F92A0
:10231400CDB7DEB76B017C01DC01CB01BF778B3D10
:102324002FE0920729E4A2072FE3B20728F50097CC
:1023340020E8A20729E3B207E0F40097A048B1051A
:1023440048F420E030E040E853E0C701B6010E94C1
:102354001B2908C020E030E040E85BE7C701B60174
:102364000E94972869837A838B839C83C701B60173
:10237400A1C0C701B60198C0B701A601442777FDE3
:102384004395552766277727823D23E592072BE758
:10239400A20720E4B20768F5843E9B4CA641B044F2
:1023A400A0F4452B49F02BED3FE049EC5FE3C70176
:1023B400B6010E9497287BC02BED3FE049EC5FE318
:1023C400C701B6010E9496286BC0452B49F02BED3E
:1023D4003FE049E450E4C701B6010E94972863C076
:1023E4002BED3FE049E450E4C701B6010E94962872
:1023F4005AC0863D21E3920722EEA20720E4B207E9
:1024040068F5803E9D4EAF4AB044A0F4452B49F098
:1024140024EE3BEC46E950E4C701B6010E9497283C
:102424003FC024EE3BEC46E950E4C701B6010E94EC
:1024340096283DC0452B49F02BED3FE049EC50E494
:10244400C701B6010E9497282FC02BED3FE049EC4D
:1024540050E4C701B6010E94962826C00097A04800
:10246400BF4738F0A7019601C701B6010E9496281C
:1024740021C0AE014F5F5F4FC701B6010E944413F4
:102484009C012370332769817A818B819C8121305F
:10249400310531F02230310531F0232B41F404C0F1
:1024A4000E947B1807C090580E94031803C00E9422
:1024B4007B1890582496CDBFDEBFDF91CF91FF905B
:0824C400EF90DF90CF90089526
:1024CC004F925F926F928F929F92AF92BF92CF92E8
:1024DC00DF92EF92FF920F931F93CF93DF9300D075
:1024EC000F92CDB7DEB76C0180E090E00E94C7265A
:1024FC0069837A838B839C83CE0101962C0120E81F
:10250C00622E862DB2010E94F5287C01FC012281ED
:10251C0033818091A42C90E02817390709F498C0D6
:10252C002093A42CA084B18401E0F2E0AF16B10496
:10253C000CF000E0F701868097806285738510E0CF
:10254C00601B710B072E000C880B990B0E94921FBD
:10255C0020E030EA46EB53E40E941B290E944D22F6
:10256C00860E971EB5016E5F7F4F5801AA0CBB1CDF
:10257C000A0D1B1D000F111F000F111F600F711F83
:10258C00072E000C880B990B0E94921F21E03DEC4A
:10259C0044EF51E40E941B290E944D22680D791DC5
:1025AC006459754C9B012227330F221F3327F601E8
:1025BC0082819381822B932B906482839383660F09
:1025CC00771FF701848095809594879495948794D0
:1025DC00959487949594879468297929F601648356
:1025EC007583F701848120E030E0382F3295307FFD
:1025FC00828193810024969587950794969587956B
:10260C000794982F802D822B932BF601868397832A
:10261C00862DB2010E94FA28FC012481F7018481E5
:10262C00281B422F022E000C550B55231CF45195E0
:10263C0041955109F60186819781842B952B8683D0
:10264C00978322233CF480628683978381E003C0C6
:10265C0080E001C081E02496CDBFDEBFDF91CF9139
:10266C001F910F91FF90EF90DF90CF90BF90AF90A4
:0C267C009F908F906F905F904F9008959A
:102688004F925F926F927F92AF92BF92CF92DF92FA
:10269800EF92FF920F931F93CF93DF93CDB7DEB7DF
:1026A8002C97CDBFDEBF2B013C015A01DC01CB01C9
:1026B800BF778B3D2FE0920729ECA2072DE4B207E4
:1026C80008F042C023E839EF42E25FE3C301B201F8
:1026D8000E941B2920E030E040E45BE40E94972838
:1026E80020E030E040E45BE40E9496286B017C0126
:1026F8000E94B22869877A878B879C872AED3FE0FA
:1027080049EC5FE3C701B6010E941B299B01AC019C
:10271800C301B2010E9496282B013C0123EA35E847
:1027280048E852E3C701B6010E941B299B01AC018E
:10273800C301B2010E949628F501608371838283E8
:10274800938389859A8552C00097F0E8AF07FFE721
:10275800BF0770F0A3019201C301B2010E9496283D
:10276800F501608371838283938380E090E03EC0AB
:10277800AC01BD0127E176956795579547952A9550
:10278800D1F746595109610971096A017B0137E19D
:10279800CC0CDD1CEE1CFF1C3A95D1F78C199D0959
:1027A800AE09BF098D839E83AF83B88700E010E030
:1027B80021E030E0BE016F5F7F4FCE0105960E9499
:1027C800A70249815A816B817C8177FE0AC07058C3
:1027D800F5014083518362837383919581959109B3
:1027E80005C0F50140835183628373832C96CDBF66
:1027F800DEBFDF91CF911F910F91FF90EF90DF9097
:10280800CF90BF90AF907F906F905F904F9008955A
:102818006F927F928F929F92AF92BF92CF92DF92E8
:10282800EF92FF920F931F93CF93DF9300D000D0C6
:10283800CDB7DEB77B013C0199231CF42FEF621A58
:10284800720A759467941D821E8281C04D815E81D3
:1028580060E0C7010E94050F69837A838B839C839C
:10286800B30180E090E00E94901F4B015C019B0146
:10287800AC0169817A818B819C810E941B299B0113
:10288800AC01C501B4010E9497280D811E81000F7B
:10289800111FF801EE54F64D6F010E944D22F6010A
:1028A800608371834D815E8161E0C7010E94050FDD
:1028B8009B01AC01C501B4010E941B299B01AC011D
:1028C800C501B4010E94972898012E5C374D690113
:1028D8000E944D22F601608371834D815E8162E022
:1028E800C7010E94050F9B01AC01C501B4010E94FC
:1028F8001B299B01AC01C501B4010E9497289801CE
:102908002E54394D69010E944D22F601608371836E
:102918004D815E8163E0C7010E94050F9B01AC01F8
:10292800C501B4010E941B299B01AC01C501B4017A
:102938000E9497280E5C1A4D0E944D22F801608370
:1029480071832D813E812F5F3F4F2D833E838D8183
:102958009E818E159F0508F479CF2696CDBFDEBFE0
:10296800DF91CF911F910F91FF90EF90DF90CF9063
:0E297800BF90AF909F908F907F906F900895CA
:102986000F931F93CF93C82F8B018E3F39F481E0AD
:102996008093A82C1092942C1092952CCF3F09F07E
:1029A6003FC02091942C3091952C2730310568F446
:1029B600A8016DE08091A92C0E94A8221092A82C53
:1029C6001092942C1092952C2BC08091092090E0A7
:1029D60006962817390739F0A80168E08091A92CD6
:1029E6000E94A82217C086E090E20E94841E8823D7
:1029F60039F0A80161E08091A92C0E94A8220AC0A2
:102A060086E090E20E944A10A801682F8091A92CC6
:102A16000E94A8221092A82C1092942C1092952C09
:102A26008091A82C813009F04AC0CE3F08F047C0FB
:102A36008091942C9091952C87309140A0F5CD3FB4
:102A460071F18091A72C8130D1F4CC2389F0C1306B
:102A560089F0C23089F01092A82C1092942C109212
:102A6600952CA8016CE08091A92C0E94A82205C093
:102A7600CDEF03C0CEEF01C0CFEF1092A72C80910F
:102A8600942C9091952C9C012F5F3F4F2093942C72
:102A96003093952CFC01EA5FFF4DC08310C081E0A6
:102AA6008093A72C0CC01092A82C1092942C1092F4
:102AB600952CA8016AE08091A92C0E94A822CF91AA
:062AC6001F910F9108951D
:102ACC001F93CF93DF93CDB7DEB78F810E9423295D
:102ADC006D968FAD6D97803218F06D961FAE6D9719
:102AEC00CE59DE4F8881C256D1408823A1F08DB7D4
:102AFC009EB7C4978DBF9EBFADB7BEB7119684E38A
:102B0C00FE01EF59FE4F01900D928A95E1F70E945C
:102B1C005B26CDBFDEBF6A968EAD9FAD6A970E94D5
:102B2C00E128CE0108960E947224CE0140960E94A4
:102B3C003F1D6D968FAD6D970E94262961968FADC6
:102B4C006197882329F0CE01805B9F4F0E947C22E5
:102B5C006C968FAD6C970E9429296B968FAD6B97F5
:102B6C000E94B32781E00E9432296E968FAD6E973A
:102B7C000E942C296F968FAD6F970E942F29A196DA
:102B8C008EAD9FADA1970E941B28A3968EAD9FADD5
:102B9C00A3970E945928A4968FADA4970E94E6286B
:102BAC0010E00BC0E4E6F0E0EC0FFD1FE10FF11DAF
:102BBC006081812F0E94C5281F5FC05ADE4F88811B
:102BCC00C056D140181770F30E943529CB56DE4FF2
:102BDC008881C559D1400E94322980EB0E94A727D9
:082BEC00DF91CF911F910895C4
:102BF4004F925F926F927F928F929F92AF92BF9209
:102C0400CF92DF92EF92FF92CF93DF93CDB7DEB7EF
:102C14002897CDBFDEBF6B017C01DC01CB0147E10E
:102C2400B695A795979587954A95D1F799278F5784
:102C34009109873191059CF597FD36C088248A94C3
:102C4400982C3FE7A32EB12C04C0B594A794979475
:102C540087948A95D2F7D501C4018C219D21AE2198
:102C6400BF21892B8A2B8B2BD1F020E030E040E868
:102C74005BE7C701B6010E9497286D837E838F832B
:102C84009887F7FE04C0C80CD91CEA1CFB1C80946E
:102C94009094A094B094C820D920EA20FB205C2D05
:102CA4004D2D3E2D2F2D21C020E030E040E85BE784
:102CB400C701B6010E94972869837A838B839C831A
:102CC400F7FE0FC0D701C601880F991FAA1FBB1FAB
:102CD400892B8A2B8B2B19F350E040E030E82FEB43
:102CE40004C050E040E030E020E0652F742F832FD3
:102CF400922F2896CDBFDEBFDF91CF91FF90EF904A
:102D0400DF90CF90BF90AF909F908F907F906F9007
:062D14005F904F9008954E
:102D1A00CF92DF92EF92FF921F93CF93DF93EC0152
:102D2A001091A22C11110FC080918C2C882359F07C
:102D3A0044EA53E260E828E030E084E79CE20E943B
:102D4A000A2410928C2C8091F62380FBCC24C0F8A4
:102D5A00D12CC60182959295907F9827807F9827DB
:102D6A004A815B819C01242B352B2A833B838091EA
:102D7A00F92380FBEE24E0F8F12CC701880F991F94
:102D8A00880F991F880F991F822B932B8A839B8305
:102D9A002091FA2343E050E0411B510930E002C080
:102DAA00359527954A95E2F721703327220F331F6D
:102DBA00220F331F822B932B1370812B8A839B83C1
:102DCA000E94BB218C839D834091A22C242F30E04A
:102DDA00220F331FF901EC58F34D808190E0982FB0
:102DEA008827F901EB58F34D2081822B8E839F832C
:102DFA0081E0840F8093A22C843011F41092A22CCB
:102E0A00DF91CF911F91FF90EF90DF90CF900895BF
:102E1A005F926F927F928F929F92AF92BF92CF9260
:102E2A00DF92EF92FF920F931F93CF93DF936B0181
:102E3A00E82EEA018091CC0188608093CC0140E2BF
:102E4A000FEF17E075E3FF24F3942115310509F418
:102E5A0048C08C2F8F71542F581B852F90E028174C
:102E6A00390708F4C901982ED6013601E0E88E2EFA
:102E7A00F801E81BF90BEC17FD0710F40E941F2953
:102E8A005091CF0157FDFCCF562C5E01F0EFBF1ACF
:102E9A006301E82C5091CF0157FDFCCFF6015E2D5E
:102EAA000E947128F50161935F01FFEFCF1ADF0AD3
:102EBA00EF0A5C2D5519591568F31092C201D09387
:102ECA00C101C093C0017093CA01F8EDF4BFF0923A
:102EDA00CB016D01C80ED91EC80FD91F281B390B8B
:102EEA00B4CF8091CC01877F8093CC01DF91CF91C1
:102EFA001F910F91FF90EF90DF90CF90BF90AF900E
:0C2F0A009F908F907F906F905F900895D3
:102F16000F931F93CF93DF938C018091902C88237E
:102F260019F081508093902C80918D2C882391F0FC
:102F36004CEA53E260E820E430E08AE99BE20E9432
:102F46000A24ECE8FCE2928181E0892782831182DF
:102F56001092A02CECE8FCE282818170C82F60E020
:102F6600D62FC295D295D07FDC27C07FDC27D062D2
:102F76004091A02C842F8F70C82BD80112968D916A
:102F86009C911397C82BD92B1296CD93DC9313974C
:102F9600842F90E0880F991F880F991FDC01A65691
:102FA600B44D2C9130E0322F2227DC01A556B44DCA
:102FB6005C91252BD80114962D933C931597DC0133
:102FC600A456B44D2C9130E0322F2227DC01A356B3
:102FD600B44D8C91B901682BCB01D80116968D930F
:102FE6009C93179781E0840F8093A02C938189137B
:102FF60002C01092A02CDF91CF911F910F910895DE
:103006004F925F926F927F928F929F92AF92BF92F2
:10301600CF92DF92EF92FF92CF93DF9300D00F9281
:10302600CDB7DEB74B015C019B01AC010E941B29A9
:103036006B017C019B01AC01C501B4010E941B29F7
:1030460069837A838B839C832CE33CE646E356E3D1
:10305600C701B6010E941B292FEC37E040E559E372
:103066000E9496282B013C01A7019601C701B601D3
:103076000E941B2929813A814B815C810E941B2970
:103086009B01AC01C301B2010E941B292B013C012B
:1030960024E838E848E05CE3C701B6010E941B2932
:1030A6002BEA3AEA4AE25EE30E94962829813A81AF
:1030B6004B815C810E941B29A50194010E949728DF
:1030C6009B01AC01C301B2010E9497282496CDBF93
:1030D600DEBFDF91CF91FF90EF90DF90CF90BF9052
:1030E600AF909F908F907F906F905F904F900895D4
:1030F6004F925F926F927F928F929F92AF92BF9202
:10310600CF92DF92EF92FF92CF93DF9300D00F9290
:10311600CDB7DEB79B01AC010E941B296B017C0178
:103126009B01AC010E941B292B013C0120E030E0F1
:1031360040E05FEBC701B6010E941B2920E030E0AA
:1031460040E85FE30E9497284B015C012FE93AEAC9
:103156004AE25DE3C301B2010E941B299B01AC0157
:10316600C501B4010E9497284B015C0127E13AE9A9
:103176004CEC57E3C701B6010E941B292FE334E04C
:1031860046EB5AE30E94962869837A838B839C8355
:10319600A3019201C701B6010E941B299B01AC0144
:1031A60069817A818B819C810E941B299B01AC01DC
:1031B600C501B4010E9497282496CDBFDEBFDF91DA
:1031C600CF91FF90EF90DF90CF90BF90AF909F9000
:0C31D6008F907F906F905F904F90089555
:1031E20010C00E94A42858F00E949D2840F029F4A3
:1031F2005F3F29F00C94D12851110C94AC280C9407
:1032020038290E942E2468F39923B1F3552391F3B0
:10321200951B550BBB27AA2762177307840738F043
:103222009F5F5F4F220F331F441FAA1FA9F335D0A0
:103232000E2E3AF0E0E832D091505040E695001C54
:10324200CAF72BD0FE2F29D0660F771F881FBB1F0E
:10325200261737074807AB07B0E809F0BB0B802DEC
:10326200BF01FF2793585F4F3AF09E3F510578F018
:103272000C94D1280C94AC285F3FE4F3983ED4F32D
:10328200869577956795B795F7959F5FC9F7880FEC
:10329200911D9695879597F90895E1E0660F771F3E
:1032A200881FBB1F621773078407BA0720F0621BCF
:0E32B200730B840BBA0BEE1F88F7E09508959E
:1032C000DC01E3E6FCE26081862F82958F7090E05E
:1032D000AC01542F44275295507F6170362F330F25
:1032E000330F330F20E0422B532B828120E1829F4A
:1032F000C0011124482B592B818190E0880F991F20
:10330000880F991F880F991F482B592B2381822FD3
:10331000869586958695482B12968D919C9113974C
:10332000482B592B12964D935C93139730E0322F14
:1033300022273295330F307E85818F7340E8849F3A
:10334000C0011124282B392B47814F7350E0440FC3
:10335000551F242B352B8481982F92959695977025
:10336000292B14962D933C93159790E0982F88273E
:10337000990F990F990F26812F7340E2249F900196
:103380001124822B932B20852F71822B16968D93DF
:063390009C9317970895BD
:103396000FC00E949D2838F00E94A42820F0952393
:1033A60011F00C94D1280C94382911240C94AC28D3
:1033B6000E942E2470F3959FC1F3950F50E0551F80
:1033C600629FF001729FBB27F00DB11D639FAA2774
:1033D600F00DB11DAA1F649F6627B00DA11D661FC3
:1033E600829F2227B00DA11D621F739FB00DA11DE4
:1033F600621F839FA00D611D221F749F3327A00D9E
:10340600611D231F849F600D211D822F762F6A2F39
:1034160011249F5750409AF0F1F088234AF0EE0F9E
:10342600FF1FBB1F661F771F881F91505040A9F7CB
:103436009E3F510580F00C94D1280C94AC285F3F38
:10344600E4F3983ED4F3869577956795B795F79507
:10345600E7959F5FC1F7FE2B880F911D969587957F
:0434660097F9089535
:10346A00CF93DF93EC018091F4239091F523888325
:10347A0099838091F7238170382F330F330F20E01F
:10348A008091F8238F7140E2849FC0011124822B1E
:10349A00932B8A839B831C821D821E821F828091AA
:1034AA003125882329F0CE010E94661281113DC080
:1034BA008091A62C8F5F8093A62C9091FC2489176B
:1034CA0010F01092A62C9091A62CE92FF0E0E05073
:1034DA00FC4D8081843179F42091EC23222321F060
:1034EA00CE010E94931D21C09F5F9093A62C9C3F02
:1034FA0010F01092A62C843069F018F4882331F069
:10350A0014C0863059F0863169F00FC0CE010E948E
:10351A008D160BC0CE010E948B1707C0CE010E94E8
:10352A00351E03C0CE010E946019DF91CF91089524
:10353A0011C00E949D2838F00E94A42820F039F476
:10354A009F3F19F426F40C9438290EF4E095E7FB12
:10355A000C94D128E92F0E942E2458F3BA17620737
:10356A0073078407950720F079F4A6F50C94AB2825
:10357A000EF4E0950B2EBA2FA02D0B01B901900184
:10358A000C01CA01A0011124FF27591B99F0593FC8
:10359A0050F4503E68F11A16F040A22F232F342F10
:1035AA004427585FF3CF469537952795A795F0405E
:1035BA005395C9F77EF41F16BA0B620B730B840B73
:1035CA00BAF09150A1F0FF0FBB1F661F771F881F2B
:1035DA00C2F70EC0BA0F621F731F841F48F4879583
:1035EA0077956795B795F7959E3F08F0B0CF939575
:0E35FA00880F08F09927EE0F97958795089592
:10360800CF9320E040EA56E861E070E080EA94E079
:103618000E94F52523E04FEF60E680EA94E00E94DF
:103628008821853009F04EC0C0E00BC020E12C0F86
:1036380040E860E680EA94E00E948821853019F429
:10364800CF5FC83098F38530E9F5C0E027C08C2FEC
:1036580090E09C01220F331F820F931F9C01092EBB
:10366800000C440B2E573B4F4F4FF901542F0E942B
:10367800FF27262F0296092E000CAA0B8E579B4F68
:10368800AF4FFC015A2F0E947128462F60E680EA4E
:1036980094E00E948821853019F4CF5FC133B8F2D5
:1036A800853081F421EB4CEA60E680EA94E00E94E0
:1036B8008821853039F423E04AEF60E680EA94E017
:0836C8000E948821CF910895B2
:1036D000EF920F931F93CF93DF936894EE24E1F85A
:1036E00000E020E040E060E280E096E00E943925C2
:1036F000E0E0F6E014E01083168340E268E080E04A
:1037000096E00E948F28C0EAD0E08A8182608A8396
:10371000EE24E39420E040E062E080E296E00E9444
:1037200039251093200642E063E080E296E00E9493
:1037300088288A8184608A83E0E4F6E088E08083D8
:1037400086830F2EF7E0EF2EF02D08E220E040E018
:1037500067E080E696E00E943925E0E6F6E087E043
:103760008083858320E040E060E480E896E00E946A
:103770003925E0E8F6E088E4808380E48483E0EAA9
:10378000F6E084EB808380E18483DF91CF911F9109
:063790000F91EF90089577
:10379600AF92BF92CF92DF92EF92FF920F931F9359
:1037A600CF93DF937C01EB01C12CD12C42C0C60123
:1037B600880F991FF701E80FF91F00811181FC019D
:1037C600E75AF34DA080B180F7018281938193FF80
:1037D60006C0F3E0CF16D10411F4A12CB12CC80118
:1037E6000E94B0248A259B2520E030E00AC0412FA4
:1037F600441F4427441F4883000F111F2F5F3F4F6C
:103806002196203131059CF320E030E00CC0BE014A
:103816006F5F7F4F41E091FF40E04883880F991F1B
:103826002F5F3F4FEB012A3031058CF38FEFC81A1B
:10383600D80AE4E0CE16D1040CF4B9CFDF91CF91CB
:103846001F910F91FF90EF90DF90CF90BF90AF90B8
:023856000895D3
:103858004F925F926F927F928F929F92AF92BF9298
:10386800EF92FF920F931F93CF93DF938B017C010D
:1038780099231CF42FEFE21AF20AF594E794C0E0BA
:10388800D0E033C0BE01C8010E94B1202B013C0129
:10389800B70180E090E00E94901F4B015C019B0102
:1038A800AC01C301B2010E941B299B01AC01C501F7
:1038B800B4010E9497280E944D229E01220F331FB7
:1038C800F901EE54F64D60837183F901EE5CF74D12
:1038D80060837183F901EE54F94D60837183F901B6
:1038E800EE5CFA4D608371832196C017D10750F2C0
:1038F800DF91CF911F910F91FF90EF90BF90AF9004
:0E3908009F908F907F906F905F904F900895EA
:103916008091982C882331F082E39BE20E9437271E
:103926001092982C8091992C882311F1E0919C2C6F
:1039360021E02E0F20939C2CF0E0EE5CF44D90815C
:1039460080919B2C8927817080939A2C80939B2C45
:1039560090919D2C990F892B837080939D2C2836EE
:1039660029F410929C2C81E08093982C1092992C2B
:1039760080919F2C882389F0E0919D2CF0E0EE0F3A
:10398600FF1FE459F34D60E0808191810E94C223BC
:1039960081E08093992C10929F2C80919E2C8823F5
:1039A60089F0E0919D2CF0E0EE0FFF1FE459F34DF6
:1039B60061E0808191810E94C22381E08093992CED
:0639C60010929E2C0895F2
:1039CC000F931F93CF93DF93EA0140385105D4F046
:1039DC0020E030E040E05FE70E941B299E012F575A
:1039EC003109203831056CF120E030E040E05FE730
:1039FC000E941B29CE5FD109C038D1051CF1CFE73D
:103A0C00D0E020C042385F4FECF420E030E040E8DA
:103A1C005CE00E941B299E012A593F4F22384FEF30
:103A2C0034077CF420E030E040E85CE00E941B2985
:103A3C00C453DF4FC2382FEFD20724F4C2E8DFEFB4
:103A4C0001C0E9019E0121583F4F8901330F220B20
:103A5C00330BA9019801E7E1220F331F441F551FB7
:103A6C00EA95D1F70E941B29DF91CF911F910F91FD
:023A7C000895AB
:103A7E00CF92DF92EF92FF920F931F93CF93DF932C
:103A8E006C0120E8E22E8E2DB6010E94A426EC01D8
:103A9E0081E080938D2C80E4ECEAF3E2DF011D924D
:103AAE008A95E9F78E01112798016E2DA601CF0197
:103ABE000E946B25BFE3BC17F8F0CF5FF801ED5500
:103ACE00FC4D8DE0818720E030E012C04C2F50E09D
:103ADE00241735075CF0C90199230CF403969595CC
:103AEE0087959595879580938F2C09C02C5F3F4FB6
:103AFE00213431055CF303C080E180938F2CECE818
:103B0E00FCE283818483DF91CF911F910F91FF900F
:083B1E00EF90DF90CF900895B5
:103B26000F931F93CF938C01C091A32CC1110FC08B
:103B36008091912C882359F04CEE53E260E828E0FE
:103B460030E08CE79CE20E940A241092912C2C2FE4
:103B56002370F80182819381822B906A82839383FA
:103B66008C2F90E0880F991F880F991FFC01E4584D
:103B7600F34D208130E0322F2227FC01E358F34D2C
:103B86004081242BF80124833583FC01E258F34D50
:103B9600208130E0322F2227FC01E158F34D80814D
:103BA600A901482BCA01F80186839783CF5FC0938A
:103BB600A32CC23011F41092A32CCF911F910F9118
:023BC600089560
:103BC80088249924F401E401B0E49F93AA279A1564
:103BD8008B049C04ED05FE05CF05D007A10798F4DA
:103BE800AD2FDC2FCF2FFE2FE92D982C892E982F63
:103BF800872F762F652F542F432F322F2227B85027
:103C080031F7BF9127C01B2EBF91BB27220F331F4F
:103C1800441F551F661F771F881F991F881C991CF2
:103C2800EE1FFF1FCC1FDD1FAA1FBB1F8A149B049A
:103C3800EC05FD05CE05DF05A007B10748F08A1899
:103C48009B08EC09FD09CE09DF09A00BB10B216027
:103C58001A94E1F62EF49401AF01BE01CD01000CD7
:023C68000895BD
:103C6A000F931F93CF93DF93CDB7DEB72597CDBFC1
:103C7A00DEBFAC01FC0122813381306322833383AE
:103C8A0002E91CE2F8019081E92FF0E0DF01AA0FB6
:103C9A00BB1FAA0FBB1FEA0FFB1FE652F44D85E0BC
:103CAA00DE01119601900D928A95E1F78981E82F3C
:103CBA00E295EF70F0E0EE0FFF1F682F617070E081
:103CCA006E2B7F2B262B372BFA01228333832C81F1
:103CDA003D81248335832A813B81268337839F5FF5
:103CEA00F80190838181981302C01092922C259634
:0E3CFA00CDBFDEBFDF91CF911F910F910895D6
:103D0800EF92FF921F93CF93DF93EC016B8115E045
:103D1800160F88818E3FF1F4E12EF12CFE01EE0D95
:103D2800FF1D319780818F3FA9F421966F5FCE01E7
:103D38000E947920EC0EFD1EF7013497208130E0B7
:103D4800322F222731964081242B82179307B1F016
:103D580080E017C06D5FCE010E947920C10FD11D90
:103D6800FE013297208130E0322F222721974881A7
:103D7800242B8217930721F080E003C081E001C063
:0E3D880081E0DF91CF911F91FF90EF900895A1
:103D96001F93CF93DF93C0E8D1E080EC8883E0E007
:103DA600F3E081E0818388E08283138285E080836B
:103DB600E0E0F1E084E8808319E5128B75E1738B0E
:103DC600C48BD58B168A22EB39E2208FC901330FBB
:103DD600AA0BBB0B892F9A2FAB2FBB27818F128E75
:103DE60068E1648F53E0558F168E45E2408B30892B
:103DF6003068308B12A373A3C4A3D5A316A220A741
:103E060081A712A664A755A716A640A380A180681D
:0A3E160080A3DF91CF911F91089562
:103E20001F920F920FB60F92112408B60F9218BE70
:103E300009B60F9219BE0BB60F921BBE2F933F937C
:103E40004F935F936F937F938F939F93AF93BF93A2
:103E5000EF93FF938091A52C882361F08091000857
:103E6000813041F480916E2290916F220E946427EC
:103E70001092A52C0E941329FF91EF91BF91AF9151
:103E80009F918F917F916F915F914F913F912F9172
:103E90000F900BBE0F9009BE0F9008BE0F900FBE83
:063EA0000F901F90189521
:103EA600E0E5F0E080818260808360E080E00E944F
:103EB600B9288091510081FFFCCF81E00E94E02566
:103EC6000E94041B40E060E080EC0E94E127E0E5F0
:103ED600F0E08081886080838091510083FFFCCF71
:103EE60083E00E94E02582E00E94EB2762E080ECFE
:103EF6000E94D728E0E5F0E080818061808360E061
:103F060080E00E94B9288091510084FFFCCF84E0B4
:0A3F16000E94E0250E94BF280895D4
:103F2000E89409C097FB3EF4909580957095619553
:103F30007F4F8F4F9F4F9923A9F0F92F96E9BB2709
:103F40009395F695879577956795B795F111F8CF85
:103F5000FAF4BB0F11F460FF1BC06F5F7F4F8F4FF0
:103F60009F4F16C0882311F096E911C0772321F0E6
:103F70009EE8872F762F05C0662371F096E8862F7E
:103F800070E060E02AF09A95660F771F881FDAF7D5
:0A3F9000880F9695879597F908951C
:103F9A001F920F920FB60F92112408B60F9218BEF5
:103FAA0009B60F9219BE0BB60F921BBE2F933F9301
:103FBA004F935F936F937F938F939F93AF93BF9327
:103FCA00EF93FF9363EA73E280E82FE831E040E081
:103FDA0050E00E940D17FF91EF91BF91AF919F9111
:103FEA008F917F916F915F914F913F912F910F9098
:103FFA000BBE0F9009BE0F9008BE0F900FBE0F9018
:04400A001F90189556
:10400E000E94681B0E94531F0E94D4220E94CB1E46
:10401E0060E070E080E00E94D826813049F42FE8FD
:10402E0031E040E050E060E084E192E20E948E27B1
:10403E008DB79EB78F5891408DBF9EBFADB7BEB79F
:10404E0011968FE891E0E4E1F2E201900D92019772
:10405E00E1F70E9466158DB79EB781579E4F8DBFB3
:10406E009EBF0E9419270E948B1C0E94F9260E9457
:04407E001F25F9CF32
:10408200EF92FF920F931F93CF93DF937C018B01EB
:10409200C0E0D0E023C0CE010E94CB289C01E29E6A
:1040A200C001E39E900DF29E900D11249E01220FFD
:1040B200331FF901EE54F64D80839183F901EE5CD2
:1040C200F74D80839183F901EE54F94D80839183FA
:1040D200F901EE5CFA4D808391832196C017D107D6
:1040E200D0F2DF91CF911F910F91FF90EF90089541
:1040F2002FEF3FEFE0E0F0E02AC0322723273227FC
:10410200DC01AE0FBF1F4C91D901A427AD019A016A
:1041120033273595279535952795359527953595E7
:10412200279524273527A901542F44275295507FDC
:1041320024273527A9015527440F551F429552952B
:10414200507F5427407F5427242735273196462F06
:1041520050E0E417F5078CF2C90180959095089517
:10416200CF92DF92EF92FF92CF93DF93EB019C010C
:10417200ABEABAEA0E944627969587959295829570
:104182008F7089279F708927BC0180E090E00E9490
:10419200901F9B01AC0166E57EE089EC90E40E94F1
:1041A20017296B017C01BE0180E090E00E94901F04
:1041B2009B01AC01C701B6010E941B290E9482111A
:0E41C200DF91CF91FF90EF90DF90CF900895A6
:1041D000A0E0B0E0EEEEF0E20C945825EA01FB011D
:1041E000582F0E9472274B015C01C12CD12C760103
:1041F0008E019B01A50160E070E080E090E00E94EC
:10420000D90C97FF09C08FE490E080930020909331
:10421000012080E090E00DC0188A198A1A8A1B8A52
:104220001C8A1D8A89E495E0A0E08E8B9F8BA88F65
:0C423000CE01CDB7DEB7ECE00C94A22567
:10423C001F920F920FB60F92112408B60F9218BE50
:10424C0009B60F9219BE0BB60F921BBE2F933F935C
:10425C004F935F936F937F938F939F93AF93BF9382
:10426C00EF93FF9384E39CE20E940A26FF91EF9167
:10427C00BF91AF919F918F917F916F915F914F9172
:10428C003F912F910F900BBE0F9009BE0F9008BE5F
:0A429C000F900FBE0F901F901895B1
:1042A6001F920F920FB60F92112408B60F9218BEE6
:1042B60009B60F9219BE0BB60F921BBE2F933F93F2
:1042C6004F935F936F937F938F939F93AF93BF9318
:1042D600EF93FF9384E39CE20E940525FF91EF9103
:1042E600BF91AF919F918F917F916F915F914F9108
:1042F6003F912F910F900BBE0F9009BE0F9008BEF5
:0A4306000F900FBE0F901F90189546
:104310000F931F93CF93DF93EC01042F122F40E0F4
:104320000E941D228330B9F08823B9F0612FCE019D
:104330000E946E268A3099F0882399F0602FCE0172
:104340000E946E268A3079F0882379F0CE010E948F
:10435000FF2885E00BC083E009C080E007C08AE049
:1043600005C080E003C08AE001C080E0DF91CF910A
:064370001F910F9108955A
:104376002091FE24222351F13091A12C31110AC043
:1043860080E090EE920F2091FF24822B3F5F3093C6
:10439600A12C13C0432F50E0FA01E150FB4D80E001
:1043A6009081FA01E050FB4D2081222311F0822BEF
:1043B60001C08D6C3E5F3093A12C3091FD2420917D
:1043C600A12C231728F01092A12C08958DEC90EEC5
:0243D600089548
:1043D800689401C0E894F92FF12B12F00C9483270C
:1043E800A0E0B0E0EAEFF1E20C945825092E05941C
:1043F80022F40E940927112392F4F0E80F26FFEF18
:10440800E094F09400951095B094C094D094A19441
:10441800BF0ACF0ADF0AEF0AFF0A0F0B1F0B0E9421
:10442800E41D07FC0E940927CDB7DEB7ECE00C9429
:02443800A225BB
:10443A00FF920F931F93CF93DF93EC01F62E042F75
:10444A000E94E926182F813021F0CE010E94E92628
:10445A0019C00230A0F46F2D70E0660F771F602B31
:10446A006E83602FCE010E942B238A3059F08C81F3
:10447A0084FF07C0CE010E94FF2880E003C084E0C9
:10448A0001C0812FDF91CF911F910F91FF90089565
:10449A000E94362488F09F5798F0B92F9927B75170
:1044AA00B0F0E1F0660F771F881F991F1AF0BA95CE
:1044BA00C9F714C0B13091F00E94AB28B1E0089559
:1044CA000C94AB28672F782F8827B85F39F0B93F4B
:1044DA00CCF3869577956795B395D9F73EF4909581
:0E44EA008095709561957F4F8F4F9F4F08957D
:1044F800CF92DF92EF9221E02093912CDC012C9156
:104508002223B9F06C0148E050E060E270E08CEEE4
:1045180093E20E943628B0E8EB2E8E2DB6010E9459
:10452800A4269C016E2DA6018CEE93E20E946B25B9
:1045380007C088E0ECEEF3E2DF011D928A95E9F707
:08454800EF90DF90CF90089581
:104550000F931F93CF93DF938150823000F58A0130
:10456000CEE4DCE28EEF8883E3E4FCE2808191819B
:1045700099838A8382818B8383E08C8388E18D8316
:104580006E8385E28F8368E0CE010E947920988750
:1045900089878FEF8A876BE0CE01F8011995DF914B
:0845A000CF911F910F910895C6
:1045A800E0E8F6E084E0828388E0818341E060EA25
:1045B8007AE084E39CE20E941228E091342CF09186
:1045C800352C83E0858383818F7C80618383A0EA97
:1045D800BAE08FEC16968C93169717961C928481E6
:1045E80080618483848188608483E0EAF0E082814A
:0845F80081608283789408952C
:10460000E894DF93CF93FC01DB010E9446277F9360
:104610006F93E9019A01AC01BF93AF933F932F933E
:10462000DF010E94462726F46C1B7D0B820B930B47
:104630009E01EB01FC010E944828AF91BF912F9190
:104640003F910E944828BE01CF01F9012F913F916F
:06465000CF91DF910895F7
:10465600DC01E0E0F0E070E01CC014969C91149739
:1046660020E430E0A901062E02C0440F551F0A942B
:10467600E2F7292F30E024233523232B09F071E0BC
:10468600E93E83E0F80748F48AE08A95F1F700C02E
:0E4696003196772311F385E008958AE00895A8
:1046A4001F920F920FB60F92112408B60F9218BEE4
:1046B4000BB60F921BBE8F93EF93FF938091030170
:1046C40080FF08C081E080939F2CE0E0F1E08381CB
:1046D40081608383FF91EF918F910F900BBE0F90B8
:0C46E40008BE0F900FBE0F901F9018959D
:1046F0001F920F920FB60F92112408B60F9218BE98
:104700000BB60F921BBE8F93EF93FF938091030123
:1047100081FF08C081E080939E2CE0E0F1E083817E
:1047200082608383FF91EF918F910F900BBE0F906A
:0C47300008BE0F900FBE0F901F90189550
:10473C00643071F018F4662331F019C0683069F0F8
:10474C006C3081F014C0FC01128221E024830895A6
:10475C0024E0FC0122831482089528E0FC012283CA
:10476C00148208952CE0FC01228314820895FC012C
:08477C00128221E0248308955C
:104784000F931F9361110EC0E0E0F1E0808F8C0164
:10479400092E000C220B330B012F122F232F33274A
:1047A400018F128E613069F4E0E0F1E080A7092EF8
:1047B400000CAA0BBB0B892F9A2FAB2FBB2781A709
:0847C40012A61F910F91089548
:1047CC00990F0008550FAA0BE0E8FEEF1616170616
:1047DC00E807F907C0F012161306E407F50798F07E
:1047EC00621B730B840B950B39F40A2661F0232B97
:1047FC00242B252B21F408950A2609F4A140A69513
:08480C008FEF811D811D08954D
:10481400CF92DF92EF926A01E62EDC012115310579
:10482400B9F0215031091196F6015E2D0E947128CC
:10483400FD01319760834FEFC41AD40AE40A611171
:10484400EDCF2A0F3B1F2A173B0711F01D92FBCF18
:08485400EF90DF90CF90089572
:10485C0057FD9058440F551F59F05F3F71F0479525
:10486C00880F97FB991F61F09F3F79F0879508950A
:10487C00121613061406551FF2CF4695F1DF08C029
:10488C00161617061806991FF1CF86957105610546
:04489C0008940895DF
:1048A000A1E21A2EAA1BBB1BFD010DC0AA1FBB1F34
:1048B000EE1FFF1FA217B307E407F50720F0A21BA6
:1048C000B30BE40BF50B661F771F881F991F1A9413
:1048D00069F760957095809590959B01AC01BD013D
:0448E000CF01089567
:1048E400CF92DF92EF926C0181E080938C2C48E0B0
:1048F40050E060E270E084EA93E20E94362880E8A7
:10490400E82E8E2DB6010E94A4269C016E2DA601D0
:1049140084EA93E20E946B25EF90DF90CF90089594
:1049240060EC70E08091FB239091FC230E940C14B6
:104934008091000881110FC0E0EAF0E08281846078
:1049440082837894E0E0F8E08BE890E086A397A374
:0C49540081E0808386830E940B29089577
:10496000AC0120E030E080E090E013C0752F771FAD
:104970007727771F440F551F91FB662760F9880F33
:10498000991F761721F069EB862761E096272F5F44
:0A4990003F4F2031310554F3089524
:10499A001F93CF93DF93EC01162F0E94F5278823EC
:1049AA0079F09D85FE01E90FF11D17839F5F9370D2
:1049BA009D87E881F98193812A819C7F922B938339
:0849CA00DF91CF911F910895C8
:1049D200833071F4E4E1F2E21082BF0180E82FE853
:1049E20031E040E050E00E940D170E9461280895D6
:1049F20063EA73E280E82FE831E040E050E00E9491
:084A02000D170E9461280895C0
:104A0A00FC0196858585981307C00190F081E02DF9
:104A1A0083818C7F838308958685DF01A80FB11D6A
:104A2A0017968C91A081B1818C9386858F5F837054
:044A3A0086870895CE
:104A3E0012C0E091962CF091972CE80FF11D608139
:104A4E0084E39CE20E94CD24882359F08091AA2C05
:104A5E008F5F8093AA2C8091AA2C9091AB2C8917F2
:044A6E0040F3089574
:104A7200EF920F93FC010E29442311F080E801C04C
:104A820080E0082B222311F080E401C080E0082B93
:104A92009FB7F8946093B000008B9FBF0F91EF9087
:024AA200089575
:104AA4002F923F924F925F926F927F928F929F923A
:104AB400AF92BF92CF92DF92EF92FF920F931F9328
:104AC400CF93DF93CDB7DEB7CA1BDB0BCDBFDEBF01
:024AD400199433
:104AD600CF92DF92EF926A01E62EDC01280F391F92
:104AE600A217B30751F0F6015E2D0E9471286D934F
:104AF6004FEFC41AD40AE40AF3CFEF90DF90CF90B9
:024B0600089510
:104B08009091932C983099F0E92FF0E09F01220FB3
:104B1800331F220F331FE20FF31FE652F44D808339
:104B280061837283438354839F5F9093932C08958A
:104B38002A88398848885F846E847D848C849B8425
:104B4800AA84B984C884DF80EE80FD800C811B8133
:104B5800AA81B981CE0FD11DCDBFDEBFED01089569
:104B6800052E97FB1EF400940E94792857FD07D064
:104B78000E94502407FC03D04EF40C9479285095D9
:0E4B88004095309521953F4F4F4F5F4F089558
:104B96000F93CF93DF930F92CDB7DEB72FB729834D
:104BA600F8941BBEFC0108ED04BF608389818FBFAA
:0A4BB6000F90DF91CF910F91089549
:104BC0000F931F93CF93C82F00E410E0F80160818A
:104BD000687F682B80E490E00E94CB25F8018081FB
:0A4BE0008C23CF911F910F910895CF
:104BEA001F93CF93DF93EC01122F0E941F2661E0DF
:104BFA00CE010E94092888E08983612FCE010E9494
:0A4C0A009E23DF91CF911F910895C2
:104C1400FC0193859F5F93708485A081B1812C9161
:104C2400981749F08385DF01A80FB11D13962C93C3
:0A4C3400938781E0089580E0089561
:104C3E00CF93DF93EC019A01AB01220F331F441F78
:104C4E00551F60E078E488EE91E00E9450242550D4
:084C5E002D83DF91CF91089531
:104C660097FB072E16F4009407D077FD09D00E9413
:104C7600472607FC05D03EF4909581959F4F0895F1
:084C8600709561957F4F0895C0
:104C8E00AA1BBB1B51E107C0AA1FBB1FA617B70764
:104C9E0010F0A61BB70B881F991F5A95A9F7809580
:084CAE009095BC01CD010895B1
:104CB600CF93DF93CDB7DEB786E090E08C0F9D1FD4
:104CC600AC0160E824E330E08DEF94E20E946B25AE
:064CD600DF91CF9108956B
:104CDC00CF93DF93EC016F8360E00E942B238A302B
:104CEC0031F08C8184FF02C080E001C081E0DF9153
:044CFC00CF910895B7
:104D000060EC70E08091FB239091FC230E94412095
:104D100080910008811103C081E0809300080E9407
:044D20000F290895BA
:104D240060EC70E08091FB239091FC230E942C1C8A
:104D340080910008811103C081E0809300080E94E3
:044D44000F29089596
:104D48009B01482FA82FCB01FC015A2F0E947128E4
:104D5800662319F00196A11DF7CF642FA901841BC2
:044D6800950B08950A
:104D6C00092E0394000C11F4882352F0BB0F40F46D
:104D7C00BF2B11F460FF04C06F5F7F4F8F4F9F4FAD
:024D8C00089588
:104D8E00FC010FB6F894A2E0B0E26D917D918D9189
:104D9E009C910FBE309721F0608371838283938341
:024DAE00089566
:104DB000CB0103D0808199270895E0ECF1E037859D
:104DC00037FDFDCF348538603487FC01E050F04F6B
:024DD000089544
:104DD200FC018481837059F0813031F4813031F4E7
:104DE200813029F083E0089581E0089582E00895FA
:104DF20008C084E39CE20E949B2764E278E20E945E
:104E0200C31484E39CE20E9451288111F2CF0895D9
:104E12006095709580959095309540955095219527
:104E22003F4F4F4F5F4F6F4F7F4F8F4F9F4F0895B1
:104E320044E063E080E191E00E94812844E063E085
:0E4E420080E291E00E9481280E94922408954F
:104E50001F920F920FB60F92112408B60F9218BE30
:0E4E60000F9008BE0F900FBE0F901F90189578
:104E6E00CF93DF93EC0184E89CE20E94351ABE01D9
:0E4E7E0084E89CE20E94CB1BDF91CF91089547
:104E8C00A29FB001B39FC001A39F700D811D11247F
:0E4E9C00911DB29F700D811D1124911D08956E
:104EAA0097FB57FF0C9401239F938F930E94012332
:0E4EBA006E1B7F0BAF91BF918A0B9B0B08956F
:104EC8001092000820E030E002C0225F3F4F281710
:0C4ED8003907D8F381E0809300080895AA
:104EE40057FD07C05BBF67917791879197911BBE70
:0C4EF40008956191719181919191089550
:104F0000689401C0E8948F929F92CF93DF930E94A0
:0C4F1000E41DDF91CF919F908F900895D9
:104F1C006068E0ECF1E0A785A7FDFDCFA485A86053
:0A4F2C00A4874050504F0C946B25F1
:104F3600FC018485DF01A80FB11D13968C91948521
:084F46009F5F937094870895AA
:104F4E00CF93C82F40E050E067ED7BE40E948425AC
:084F5E00C093632CCF9108956C
:104F66008093F623813011F0833019F40E940329CF
:084F760008950E940729089527
:104F7E000024A7FD00942A0F301D401D501D601DFA
:084F8E00701D801D901D0895A7
:104F96000E944627A59F900DB49F900DA49F800D5B
:064FA600911D1124089585
:104FAC00EC010E9440290E943F29CE010E94412918
:064FBC00CE010E943D2918
:104FC200662311F090E201C090E0892B482B4093B8
:044FD20052000895EC
:104FD600E0E5F0E09081282F209592239083908140
:044FE600892308957E
:104FEA00FC0195859F5F9370268581E0921301C02D
:044FFA0080E00895B6
:104FFE0057FD05C05BBF679177911BBE0895619108
:04500E0071910895FF
:10501200613019F4FC011382089524E0FC0123831A
:025022000895EF
:10502400FC01608371834283148613861686158679
:025034000895DD
:105036008093FB239093FC2360EC70E00E940C1499
:025046000895CB
:105048008093962C9093972C6093AB2C1092AA2C5B
:025058000895B9
:10505A00EE0FFF1F881F8BBF0790F691E02D1BBE36
:02506A00199497
:10506C00FC01480F591FE417F50711F06193FBCFB2
:02507C00089595
:10507E002A0D3B1D4C1D5D1D6E1D7F1D801F911F3A
:02508E00089583
:105090000E944627460F571FC81FD91F08F4319694
:0250A000089571
:1050A200FC012385948581E0291301C080E00895E5
:1050B2008093FD239093FE2381E08093A52C089595
:1050C20088ED84BF81E08093790080E090E00895CC
:1050D200B7FF0C94CB270E94CB27821B930B08951A
:1050E20057FD04C05BBF67911BBE089560810895A0
:1050F20090958095709561957F4F8F4F9F4F089542
:0E510200FC019181907F692B462B418308951B
:0E511000FC0181858C7F682B618742870895A2
:0E511E00FC018185837F682B6187438708959C
:0E512C005058BB27AA270E949D1A0C94B62645
:0E513A0000240A941616170618060906089592
:0E51480000240A941216130614060506089594
:0E515600E894BB2766277727CB0197F90895C9
:0E5164000E944D226894B1110C94AC2808955D
:0C517200682B81E490E00E94CB2508959A
:0C517E0063E083E590E00E94CB250895DB
:0C518A00E82FF0E0E050FC4D6083089539
:0C51960091E080FD90E0892F90E00895EA
:0C51A20097F99F6780E870E060E00895D6
:0A51AE006F71862B80935500089561
:0A51B800109200080E940F290895CC
:0A51C2008093F4239093F5230895E1
:0A51CC008093FF238093A92C08951F
:0A51D6000E94E62308F481E008952A
:0A51E0000E94E62308F48FEF089503
:0A51EA0042E05CE20E94E820089514
:0A51F4004BE15CE20E94E820089500
:0851FE0023E0FC012383089566
:0852060084E080936606089520
:08520E0084E080936506089519
:0852160082E080936606089512
:08521E0082E08093650608950B
:0852260081E080936606089503
:08522E000E94F1180C94B62651
:085236000E94CB190C94B6266E
:08523E008FEF9FEF0E943D2954
:065246008093A3230895EC
:06524C008093F823089591
:065252008093F72308958C
:065258008093F923089584
:06525E008093FA2308957D
:065264008093312508953E
:06526A008093FC2408956E
:065270009FEF80EC0895A1
:045276000C94000094
:04527A000E94BB01D2
:02527E00089591
:0252800008958F
:0252820008958D
:1052840001444947494C494E4552445320656E6395
:105294006F64657220402044696769746F6E20539F
:1052A400797374656D730000000000000000000055
:1052B40000000000000000000000000000000000EA
:1052C4000000000000000000004F7269656E740069
:1052D40000017101010A0101FF0F00000200040630
:1052E4001416000000000000000000000000000090
:1052F40000000000000000000000000000000000AA
:105304000000000000000000000000000000000099
:105314000000000000000000000000000000000089
:105324000000000000000000000000000000000079
:105334000000000000000000000000000000000069
:105344000000000000000000000000000000000059
:105354000000000000000000000000000000000049
:105364000000000000000000000000000000000039
:105374000000000000000000000000000000000029
:105384000000000000000000000000000000000019
:105394000000000000000000000000000000000009
:1053A40000000000000000000000000000000000F9
:1053B40000000000000000000000000000000000E9
:1053C40000000000000000000000000000000000D9
:1053D400000000000000000000060402A5AA00006E
:1053E40000000000000000000000000000000000B9
:1053F40000000000000000000000000000000000A9
:0F54040000000000000000000000000000000099
:0A541300FC0098016801B401500389
:08541D00B2293228B226322523
:015425000185
:015426000184
:00000001FF
